:100000000C9462000C94D21A0C94FF1A0C948A007F
:100010000C948A000C948A000C948A000C948A0038
:100020000C948A000C948A000C948A000C948A0028
:100030000C948A000C94BF060C948A000C948A00DD
:100040000C942C1B0C948A000C947F1E0C94BA1EEA
:100050000C948A000C948A000C948A000C948A00F8
:100060000C9443050C948A00000000002400270033
:100070002A0000000000250028002B0000000000DE
:1000800023002600290004040404040404040202DA
:100090000202020203030303030301020408102007
:1000A0004080010204081020010204081020000012
:1000B0000007000201000003040600000000000029
:1000C0000000622011241FBECFEFD8E0DEBFCDBFFD
:1000D00012E0A0E0B1E0EAECF2E402C005900D927B
:1000E000AC3BB107D9F714E0ACEBB2E001C01D9214
:1000F000A63AB107E1F710E0C4ECD0E004C02297C3
:10010000FE010E945F21C23CD107C9F70E94A720CF
:100110000C9463210C940000FB01DC0102C00190EF
:100120000D9241505040D8F708958091BC02813023
:1001300019F482E08093BC028091BC02833019F4F0
:1001400084E08093BC020895E3E0F0E089E08093CE
:100150005700849190E08670863009F491E0892FF1
:1001600008951F93182F0E94A400882379F09FB749
:1001700081E08093EC03F894A89588E18093600077
:1001800010936000112309F0A8959FBF1F91089557
:10019000382F20E08091ED039091EE038227932782
:1001A00040E061E270E19C01220F331F97FF04C021
:1001B000C9018627972701C0C9014F5F483099F7C9
:1001C0009093EE038093ED0308958436910520F417
:1001D000BC0180E090E025C08E3B910550F48A552B
:1001E0009040BC0180E090E02AE030E040E050E048
:1001F00016C0823D910550F4845B9040BC0180E0C4
:1002000090E024E630E040E050E009C08D5C904092
:10021000BC0180E090E028E532E040E050E00E9440
:10022000B62024E630E040E050E00E94B620089579
:1002300090E08C599F4F0E94E5000895DC0198964C
:10024000EC91F0E0E770F070EC55FD4F808108957F
:10025000FC0120A530E0C9018170907001962770E3
:10026000307035952795820F931F880F880F08955A
:100270008F929F92AF92BF92CF92DF92EF92FF92B6
:100280000F931F938C010E941E01D80197962C9109
:1002900030E043E150E0249FF001259FF00D349FB2
:1002A000F00D1124E051FE4F80809180A280B38038
:1002B00090E00F96AA2797FDA095BA2FBC01CD011B
:1002C00020E43FE14DE750E00E94B620A5019401F3
:1002D0000E94E92069017A0180ED97E0A0E0B0E09A
:1002E000C80ED91EEA1EFB1ED80198968C91887103
:1002F00081F060E07EEE8AEB9BE0A50194010E9414
:10030000E92028513C4F4F4F5F4FC20ED31EE41ED1
:10031000F51E87EE93E0A0E0B0E0C80ED91EEA1EFD
:10032000FB1EC701B60128EE33E040E050E00E941A
:10033000E920CA01B90128EE33E040E050E00E9414
:10034000B6201F910F91FF90EF90DF90CF90BF905C
:10035000AF909F908F9008951F93182FDB01FA01A3
:10036000482F469530E0848190E083709070982FFC
:1003700088272081820F911D11969C938E938481F2
:1003800090E08C70907076E0880F991F7A95E1F775
:100390002181820F911D13969C938E9312978481D5
:1003A00090E08073907064E0880F991F6A95E1F780
:1003B0002281820F911D15969C938E9314978481B0
:1003C00090E0807C9070880F991F880F991F23817F
:1003D000820F911D17969C938E93169735961896BB
:1003E0003F5F431708F0BFCF10FF50C08081829558
:1003F00086958695837090E02DE431E0AC01429FB4
:10040000C001439F900D529F900D11240C961196A0
:100410009C938E93808190E044E0969587954A95D1
:10042000E1F783709070AC01429FC001439F900D33
:10043000529F900D11240C9613969C938E931297B5
:10044000808190E0969587959695879583709070BA
:10045000AC01429FC001439F900D529F900D11240B
:100460000C9615969C938E931497808190E08370E0
:100470009070AC01429FC001439F900D529F900D20
:1004800011240C9617969C938E9316971F9108959E
:1004900023E08032920718F420E030E026C023E009
:1004A000883E920748F49C012F51334054E0369522
:1004B00027955A95E1F719C027E0803D920720F46F
:1004C0009C012C5D334011C028E08839920718F058
:1004D0002FEF33E00AC09C01285C374044E036959A
:1004E00027954A95E1F72D503C4FC90108958C306E
:1004F000910548F49C0174E0220F331F7A95E1F7CF
:10050000285D3C4F17C023E0843F920720F49C01F4
:1005100024523C4F0FC024E08030920718F020E9AD
:1005200038E008C09C012657334F64E0220F331F88
:100530006A95E1F7C90108959C01369527952575BF
:100540003575821B930B9C0136952795369527951B
:100550002373337383739373280F391FC901E4E046
:1005600096958795EA95E1F7820F931F8F709F709C
:1005700021E031E0AC01429FC001439F900D529FAA
:10058000900D1124892F0895882339F05F98000079
:10059000289A00005F9A000008955F98000028984C
:1005A00000005F9A000008955F9A000083B15F9891
:1005B000000090E096958795817008950F931F93A2
:1005C000082F5C9A5F985C9810E0802F80780E94DA
:1005D000C402000F1F5F1830C1F75F981F910F9181
:1005E00008958F770E94DE0208950F931F93082FBE
:1005F00010E0802F80780E94C402000F1F5F183027
:10060000C1F75F981F910F9108950F931F935F9803
:1006100080E000E0182F110F0E94D402810F0F5FBD
:100620000830C1F71F910F9108950E94F1020E94B6
:1006300005035C9A08951F93162F80680E94DE02BE
:10064000812F0E94F5025C9A1F9108951F931091CB
:10065000E1021827E8EDF2E0E80FF11D89E7678570
:100660000E941B038DE3612F0E941B0382E4612F14
:100670000E941B031F91089586E20E9415030895AE
:100680000F931F938BE20E941503082F8CE20E94A8
:100690001503282F30E096E0369527959A95E1F7D7
:1006A00010E0000F111F000F111F202B312BC9016B
:1006B0001F910F9108950F931F938C018CE1F80106
:1006C00064810E941B038DE1F80165810E941B0378
:1006D0008EE1F80166810E941B0380E2F8016781C8
:1006E0000E941B0381E2F80160850E941B0382E2E5
:1006F000F80161850E941B0383E2F80162850E9474
:100700001B0384E2F80163850E941B0385E2F80164
:1007100064850E941B038AE2F80165850E941B0321
:100720008EE6F80166850E941B038FE6F801678557
:100730000E941B0380E7F80160890E941B0381E788
:10074000F80161890E941B0382E7F80162890E9417
:100750001B031F910F910895EF92FF920F931F9328
:10076000CF93DF937B018C01603028E372072CE983
:1007700082072CE1920728F520E836E948E950E0A5
:100780000E94E920E9016897B90180E090E020E843
:1007900039E647E65FEF0E94B6206E0D7F1D801F91
:1007A000911F32E0660F771F881F991F3A95D1F786
:1007B00021E732E040E050E00E94E920890180E436
:1007C00021C020E03DE241E351E00E94E920E9013F
:1007D0006897B90180E090E020E033ED4EEC5EEFE9
:1007E0000E94B6206E0D7F1D801F911F660F771F20
:1007F000881F991F21E732E040E050E00E94E92085
:10080000890180E69E012F71622F680F85E70E94A3
:100810001B0386E7612F0E941B0387E7602F0E945E
:100820001B03CDB7DEB7E6E00C944E219F92AF924A
:10083000BF92CF92DF920F93DF93CF9300D000D07F
:10084000CDB7DEB7982E83E00E9415038093010395
:1008500084E00E9415038093020386E060E00E941A
:100860001B0387E061E00E941B0389E06FE70E94A1
:100870001B038AE065E00E941B038BE062E10E949B
:100880001B038CE065E10E941B038DE06DEF0E946D
:100890001B038EE060E00E941B03992019F08FE497
:1008A00092E008C08091FF0223E1829FC0011124E1
:1008B00080519E4F0E945B0380E36CE80E941B0303
:1008C00082E36FE00E941B0383E362E40E941B0348
:1008D00084E36AE00E941B0385E36AE20E941B0333
:1008E00086E36DE20E941B0387E364ED0E941B0315
:1008F00088E360E00E941B0389E360E00E941B0321
:10090000992049F065E8A62E61ECB62E61ECC62E62
:100910006EEDD62E08C0A090E102B090E202C09029
:10092000E302D090E4020AE38D2D9927AA27BB2782
:1009300089839A83AB83BC83802F69810E941B03C8
:10094000802F8B5F69810E941B03DC2CCB2CBA2C7F
:10095000AA240F5F0E3341F783E46FEF0E941B035D
:1009600084E46FEF0E941B0385E46FEF0E941B037A
:1009700086E46FEF0E941B03992019F08DE666E074
:1009800003C08DE66091E5020E941B0389E760E0E9
:100990000E941B038AE76091E6020E941B0383E723
:1009A00060E00E941B0384E760E00E941B03992023
:1009B00029F060EC72E98DEE99E108C06091DD02EA
:1009C0007091DE028091DF029091E0020E94AC0300
:1009D0000F900F900F900F90CF91DF910F91DF90BC
:1009E000CF90BF90AF909F90089587E061E00E9404
:1009F0001B038EE764E20E941B0388E063E00E9411
:100A00001B0388E060E00E941B0387E065E00E9412
:100A10001B0385E062E00E941B0383E00E94150334
:100A20008093010384E00E941503809302030895DC
:100A300090E0411191E0880F982B9093BA00660FD7
:100A40006093BD0030930803209307030895882323
:100A500011F085EC01C085E88093BC00089585ED18
:100A60008093BC008091BC0084FDFCCF089585EC90
:100A70008093BC000895ECEBF0E0108285E4808365
:100A800010920D0308951F920F920FB60F9211242A
:100A90002F933F934F935F936F937F938F939F9386
:100AA000AF93BF93EF93FF93DF93CF930F92CDB7A5
:100AB000DEB78091B90090E0887F90708036910514
:100AC00009F4EAC081369105CCF58832910509F424
:100AD0007CC089329105B4F48031910509F470C06D
:100AE000813191053CF4009709F40EC1089709F093
:100AF0000DC166C08831910509F467C0809709F07F
:100B000005C177C08034910509F490C08134910506
:100B100044F48033910509F46EC0C89709F0F6C01B
:100B20006CC08035910509F471C08835910509F4D0
:100B300083C08834910509F0E9C0A5C088399105C2
:100B400009F4DCC089399105ECF48837910509F482
:100B5000A3C0893791054CF48836910509F49CC0EF
:100B60008037910509F0D2C097C08838910509F403
:100B7000C5C08039910509F492C08038910509F00B
:100B8000C5C08DC0803B910509F4A5C0813B91058E
:100B90004CF4803A910509F499C0883A910509F01E
:100BA000B5C099C0803C910509F4AAC0883C910564
:100BB00009F4A6C0883B910509F0A8C080E08CC06C
:100BC000809109038093BB009BC080910C038150EE
:100BD00080930C038F5F09F43FC0E0910A03F0910A
:100BE0000B0381918093BB00F0930B03E0930A0306
:100BF00087C082E049C083E047C084E080930E0351
:100C000080910D038B7F80930D0362C08091BB00A8
:100C1000E0910A03F0910B038193F0930B03E093AF
:100C20000A0380910C03815080930C0380910C0384
:100C3000823008F065C062C08091BB00E0910A0379
:100C4000F0910B038193F0930B03E0930A038091DF
:100C50000C03815080930C0380910D038B7F809354
:100C60000D0380910D0380FF4FC080910D038E7F97
:100C700080930D0380910D03826080930D0384EABD
:100C80008093BC0043C085E080930E0380910D03E8
:100C90008B7F80930D0338C010920C0331C0E0911C
:100CA0000703F0910803309749F19091BB008091C0
:100CB0000C038F5F80930C03815011F060E001C042
:100CC00062E09983CE01019609951BC00E942F0511
:100CD0000E9437051BC081E0E0910703F0910803F3
:100CE000309761F0882311F461E001C063E0CE0128
:100CF0000196099599819093BB0003C080E001C0E3
:100D000081E00E94270502C00E942F050F90CF911D
:100D1000DF91FF91EF91BF91AF919F918F917F9163
:100D20006F915F914F913F912F910F900FBE0F9058
:100D30001F90189525B190E0FC01EE0FFF1FE80F02
:100D4000F91FEC58FC4F8081282B25B988B191817F
:100D5000892B88B98BB19281892B8BB9089585B184
:100D60009091A403892385B988B19091A503892323
:100D700088B98BB19091A60389238BB908951F92EE
:100D80000F920FB60F9211241F932F933F934F93FF
:100D90005F936F937F938F939F93AF93BF93CF9303
:100DA000DF93EF93FF931091470380918602C091E8
:100DB0008402D0918502181708F05BC08091A703C8
:100DC0009091A8039093870080938600E12FF0E034
:100DD000EE0FFF1FEE59FD4F808191810E94770237
:100DE000880F991F9093A8038093A7038091A7036E
:100DF0009091A8039E01281B390BC90130938502ED
:100E0000209384022091D3023091D402220F331F09
:100E10008217930720F430938502209384028091F7
:100E20004903882339F48091CB0280FF59C01830E0
:100E300008F456C08FEF9FEF90938B0080938A0049
:100E400080918400909185008097D0F30E94AF0636
:100E500080914803882339F480914703882319F04F
:100E600081500E949A06809147038F5F80934703C9
:100E70003EC08091A7039091A80390938700809330
:100E80008600D093A803C093A703809149038823C9
:100E900019F08FEF9FEF06C08091A7039091A803F0
:100EA0008855924090938B0080938A0080E49CE95F
:100EB00090938502809384028091840090918500B4
:100EC0008097D0F30E94AF0680914803882329F4CD
:100ED0008091860281500E949A061092470307C0B3
:100EE0008091A7039091A80388559240A5CFFF91C8
:100EF000EF91DF91CF91BF91AF919F918F917F91B2
:100F00006F915F914F913F912F911F910F900FBE65
:100F10000F901F90189590E0880F991F880F991FC8
:100F20008C30910518F42CE030E007C09C0183E080
:100F3000253F380710F024EF33E0C90108950F93DF
:100F40001F930091CC020033C0F4202F30E0C90180
:100F500080739070009719F0409749F403C0809116
:100F6000410307C0809146038295807F02C0809133
:100F7000400389010F70107016C00F33E8F410E0C1
:100F80000F701070809146038295807F0E948B07BE
:100F9000F801EE0FFF1FEE59FD4F918380830F5F25
:100FA0001F4F809140030E948B07000F111F0E59A5
:100FB0001D4FF801918380831F910F9108951F9316
:100FC00080914B0390914C038F5F9F4F39F11091AB
:100FD000CC02412F50E04F705070BA016F5F7F4FCD
:100FE000ABE4B3E020E030E02417350789F02617A2
:100FF000370711F4103360F4F8948D919C91119798
:10100000F901EE0FFF1FEE59FD4F91838083789415
:101010002F5F3F4F12962031310531F71F91089510
:101020001F93CF93DF93EC0170E0CB01827090703F
:1010300060FF1AC0892B31F080916D038883109274
:10104000EB0345C01091EB0388ED92E00E941E0176
:101050001817D8F5E12FF0E0E755FC4F8081888321
:101060001F5F1093EB0333C0892BC1F098819093DD
:10107000EA031092EB03892F807E803651F4809131
:101080006D03823010F188818F7180932B0383E090
:101090001AC09E3FE1F410926D0317C08091EA03DD
:1010A0008F3FA9F42091EB03293278F4E22FF0E08E
:1010B000E852FD4F88818083822F8F5F8093EB03FE
:1010C000893229F481E080936D0380E001C081E0E2
:1010D000DF91CF911F910895EF92FF920F931F938D
:1010E000CF93DF9380E260E040E020E138E00E94AF
:1010F000180510926D0392E0E92E85E0F82E04E0C9
:1011000080916D03813039F480E00E941604E092F2
:101110006D032D98F5CF10916D03133061F42C9869
:1011200080912B030E9426031093BC020E94F504B9
:1011300000936D03E5CF80916D03843009F78091B2
:10114000BC028430E9F68FE70E94F102C0E0D0E0F3
:1011500007C00E940503FE01E755FC4F80832196DE
:1011600088ED92E00E941E0190E0C817D9078CF329
:10117000F0926D032C9AC4CFA0E0B0E0E2ECF8E06E
:101180000C942E21EC010E94821B5B016C017E01FC
:1011900000E010E011C0209779F00E94821B6A19CC
:1011A0007B098C099D09E616F7060807190720F444
:1011B0000E943B0581E008C080910D0382FDEBCFCA
:1011C00080910E0310920E03CDB7DEB7EAE00C94C7
:1011D0004A21A0E0B0E0EFEEF8E00C943021182FA7
:1011E0007B01042FC22FD0E024E0C22ED12CCC22D0
:1011F000DD22C2FF03C080E090E004C08091820243
:10120000909183020E94BC08282F8823B9F5109280
:101210000E0300930C03F0920B03E0920A03110FEC
:1012200011601093090390910D03C1FD02C084E089
:1012300001C085E0892B80930D0380910D0381FF10
:101240000BC080910D038D7F80930D038091090366
:101250008093BB0085EC01C085EE8093BC00C0FF8D
:101260000DC0C114D10419F080E090E004C0809159
:101270008202909183020E94BC08282F822FCDB752
:10128000DEB7E8E00C944C21A0E0B0E0EAE4F9E03D
:101290000C943021182F7B01042FC22FD0E034E0B2
:1012A000C32ED12CCC22DD2222FF03C080E090E0AF
:1012B00004C080918202909183020E94BC08282F72
:1012C0008823B1F510920E0300930C03F0920B03E8
:1012D000E0920A03110F1093090390910D03C1FDD1
:1012E00002C084E001C085E0892B80930D038091CA
:1012F0000D0381FF0BC080910D038D7F80930D0343
:10130000809109038093BB0085EC01C085EE80933A
:10131000BC00C0FF0DC0C114D10419F080E090E002
:1013200004C080918202909183020E94BC08282F01
:10133000822FCDB7DEB7E8E00C944C218091BC023F
:10134000813011F081E008950E94821B20910303F7
:10135000309104034091050350910603621B730B07
:10136000840B950B615A76488140904010F480E0E0
:10137000089582E00895FF920F931F93CF93DF9318
:10138000182F092FF62E8EE30E941B03212F302FDA
:10139000C901EC0110E005C08FE769910E941B03B1
:1013A0001F5F1F15C8F385E064E00E941B0383E004
:1013B0000E9415038093010384E00E94150380932B
:1013C00002030E94821B60930303709304038093C3
:1013D00005039093060387E069E00E941B0381E008
:1013E0008093BC02CDB7DEB7E5E00C944F210E949C
:1013F000BB098091BC028130D9F40E94821B2091EC
:101400000303309104034091050350910603621BCE
:10141000730B840B950B605A76488140904040F4E2
:10142000E8CF84E894E060E071E00E946A1E0895CD
:101430008091BC028130A9F30895A1E0B0E0E3E21D
:10144000FAE00C94362180916D038230B9F480E289
:10145000BE016F5F7F4F41E021E00E94E9088823D1
:1014600079F08FEF80936D030E94741B60936E037D
:1014700070936F0380937003909371038FEF01C09B
:1014800089812196E2E00C945221A1E0B0E0EBE4E6
:10149000FAE00C94362180916D038230D9F480916A
:1014A0002B03805A898380E2BE016F5F7F4F41E04A
:1014B00021E00E944409882369F08FEF80936D0337
:1014C0000E94741B60936E0370936F03809370038C
:1014D000909371032196E2E00C945221AAE2B0E0CD
:1014E000E4E7FAE00C9434218FEF8983DE01129651
:1014F000E8EDF2E089E201900D928150E1F780E29F
:101500008E010F5F1F4FB8014AE221E00E9444099B
:10151000882351F480E2B80141E021E00E94E9080B
:10152000882311F482E001C08FEF80936D038091D6
:101530006D03823051F00E94741B60936E037093B0
:101540006F038093700390937103AA96E4E00C9468
:101550005021A2E0B0E0EFEAFAE00C9432210E94C0
:10156000821B9B01AC0180910F0390911003A0910D
:101570001103B091120379018A01E81AF90A0A0BE2
:101580001B0BD801C70181519742A040B04008F41D
:1015900044C0809113038F5F80931303815080FDBB
:1015A00002C000E001C007E020930F033093100356
:1015B000409311035093120384E894E063E00E9487
:1015C000222084E894E061E00E94222077E0F72E58
:1015D000F00E802F90E0880F991F9C012E593D4FEF
:1015E0003A832983F90160817181672F77276370BE
:1015F0007070880F991F682B792B84E894E00E9403
:101600002220E981FA8160817181707084E894E020
:101610000E9422200F5F0F15E1F62296E6E00C945F
:101620004E211F93182F84E894E0612F0E942220FE
:10163000812F0E94C8001F910895A0E0B0E0E3E26E
:10164000FBE00C943021082F0E94821B9B01AC010F
:1016500080910F0390911003A0911103B091120398
:1016600069017A01C81AD90AEA0AFB0AD701C60138
:1016700081519742A040B04008F443C020930F032B
:101680003093100340931103509312031092EE0312
:101690001092ED0388EA0E94110B002311F481E0FF
:1016A00001C081E80E94110B80E10E94110BC0E093
:1016B000D0E0FE01EE0FFF1FEE59FD4F80819181BA
:1016C0000E9477028C01E3E0000F111FEA95E1F719
:1016D000812F0E94110B802F0E94110B2196C03187
:1016E000D10539F76091EE0384E894E00E9422204E
:1016F0006091ED037091EE03707084E894E00E94B5
:101700002220CDB7DEB7E8E00C944C21A0E0B0E099
:10171000ECE8FBE00C943021182F062F0E94821B6E
:101720009B01AC0180910F0390911003A0911103D4
:10173000B091120369017A01C81AD90AEA0AFB0AB0
:10174000D701C60181519742A040B04008F4D6C1EC
:1017500020930F033093100340931103509312030F
:101760008091620290916302880F991F8093140305
:10177000977080911503887F892B809315032091A2
:10178000640230916502220F331F922F990F990F37
:10179000990F8770892B80931503422F42954695A8
:1017A000477080911603807C932F9770990F990F43
:1017B000990F842B892B8093160320916602309118
:1017C0006702220F331F922F9295990F990F907CE9
:1017D0008F73892B80931603932F9295990F990FEE
:1017E000907C822F86958695892B80931703932F63
:1017F000969596959170809118038E7F892B809392
:1018000018032091680230916902220F331F922F32
:10181000990F8170892B80931803422F441F44270E
:10182000441F80911903807F932F9770990F842B09
:10183000892B8093190320916A0230916B02220F49
:10184000331F922F9295907F8F70892B809319036D
:10185000422F42954F7080911A038078932F977092
:101860009295907F842B892B80931A0320916C0290
:1018700030916D02220F331F8F7780931A03932FBD
:10188000979599279795822F8695892B80931B038F
:10189000932F9695937080911C038C7F892B809356
:1018A0001C0340916E0250916F02440F551F942FFC
:1018B000990F990F8370892B80931C03942F929515
:1018C00096959695937020911D03207E852F8770A5
:1018D000880F880F292B282B20931D0380917002DD
:1018E00090917102880F991F382F3295330F307EF7
:1018F0002F71232B20931D03292F2295220F207E49
:10190000869586958695822B80931E038091720220
:1019100090917302880F991F80931F039770809195
:101920002003887F892B80932003209174023091BB
:101930007502220F331F922F990F990F990F8770FD
:10194000892B80932003422F4295469547708091C2
:101950002103807C932F9770990F990F990F842BF7
:10196000892B809321032091760230917702220FF8
:10197000331F922F9295990F990F907C8F73892B1B
:1019800080932103932F9295990F990F907C822F2A
:1019900086958695892B80932203932F969596950D
:1019A0009170809123038E7F892B80932303209154
:1019B000780230917902220F331F922F990F817094
:1019C000892B80932303422F441F4427441F809177
:1019D0002403807F932F9770990F842B892B8093FA
:1019E000240320917A0230917B02220F331F922F21
:1019F0009295907F8F70892B80932403422F42957C
:101A00004F70809125038078932F97709295907FE7
:101A1000842B892B8093250320917C0230917D02B9
:101A2000220F331F8F7780932503932F9795992744
:101A30009795822F8695892B80932603932F9695D1
:101A40009370809127038C7F892B8093270340918B
:101A50007E0250917F02440F551F942F990F990FCA
:101A60008370892B80932703942F92959695969552
:101A7000937020912803207E852F8770880F880F10
:101A8000292B282B2093280380918002909181029A
:101A9000880F991F382F3295330F307E2F71232BEB
:101AA00020932803292F2295220F207E8695869544
:101AB0008695822B80932903112311F490E001C0B5
:101AC00098E0002311F480E001C084E0892B80932A
:101AD0002A0384E894E06FE00E942220C4E1D3E06E
:101AE00084E894E069910E94222083E0CB32D807F9
:101AF000B9F784E894E060E00E942220CDB7DEB719
:101B0000E8E00C944C211F93182F8091C0028B3277
:101B100021F48EE0612F0E947D1C8091BF028732EC
:101B200059F4112321F08091B000806103C08091AD
:101B3000B0008F7E8093B0001F9108958091440380
:101B4000909145039F770E949C02982F80934603B3
:101B50008F3029F4809140038695805804C089E035
:101B6000989FC001112480934103F8940E949F071D
:101B700078948091BF028132C9F490914103892FFA
:101B800081508E3F60F08091B0008F7D8093B000D7
:101B900060E0911161E083E00E947D1C08959093C4
:101BA000B4008091B00080628093B00008951F93CC
:101BB000182F811111E082E1612F0E947D1C83E1C9
:101BC000612F0E947D1C10920C0310920D038091D6
:101BD000B9008C6F8093B90080E28093B80085E4EF
:101BE0008093BC001F910895CF93DF9384E894E025
:101BF0000E94AF1F892BF9F08091E803C82FD0E035
:101C00009E012F5F3F4F2F7130708091E70390E06E
:101C10002817390781F084E894E00E94E91FC9532E
:101C2000DC4F88838091E80390E001968F7190707B
:101C30008093E803DBCFDF91CF910895EF92FF927D
:101C40001F93CF93DF9388ED92E00E942801482FE5
:101C5000809386025091CC02252F30E02F70307097
:101C600090E02817390719F44F5F409386025053CC
:101C70005F3058F440918602842F90E00197281736
:101C8000390719F44F5F40938602809186028131B3
:101C900018F080E180938602E4E7F3E0108211827D
:101CA0001282339623E0E938F207C1F78FEF809371
:101CB000A4038093A5038093A6038EEBE82E82E015
:101CC000F82EAFE8B2E0E7016FEF5FEF4FEF8881EA
:101CD0008031F0F490E03C91FC01EE0FFF1FE80F23
:101CE000F91FEC58FC4F8081832B808311962C9137
:101CF00011978181822B818312969C911297828108
:101D0000892B828330954323209552239095692314
:101D10002196139682E0C53CD807C9F66093A603C6
:101D20005093A5034093A403C8E8D2E010E0F70164
:101D30008081823238F08632B0F0863219F48881A0
:101D400060E00FC0153021F48091C1008F7E05C086
:101D5000163029F48091C100877F8093C10088816B
:101D600061E00E94111C1F5F0894E11CF11C219688
:101D70001730E9F68091BE02803231F48AE061E0EA
:101D80000E947D1C82E201C082E08093800081E09D
:101D900080934803809349038091BF02813211F000
:101DA0008732D9F483E061E00E94111C83E060E097
:101DB0000E947D1C8091BF02813231F481E08093CA
:101DC000B0008093B10009C082E08093B00085E04C
:101DD0008093B1008EE38093B3008AE18093810009
:101DE0008FEF9FEF90938B0080938A0080ED97E0B8
:101DF000909387008093860080E49CE9909385020D
:101E0000809384029093A8038093A70310924703C2
:101E100080916F00816080936F008091CB0283FF7F
:101E20000DC080914B0390914C038F5F9F4F31F019
:101E30000E94DF071092490310924803DF91CF916F
:101E40001F91FF90EF90089589E060E00E94111CBF
:101E500088E061E00E94111C87E061E00E94111C93
:101E600082E060E00E94111C84E061E00E94111C8D
:101E7000089583E00E9415038093010384E00E948B
:101E800015038093020387E061E00E941B036AE070
:101E900070E080E090E00E94A81B0E94F504000022
:101EA00008950F931F93082F17C02D9A64E670E0D2
:101EB00080E090E00E94A81B2D9864E670E080E02E
:101EC00090E00E94A81B1F5F101778F36CE271E08E
:101ED00080E090E00E94A81B10E0F6CF482F392F39
:101EE00025E00DC0F999FECF1FBA842F932F92BD24
:101EF00081BD60BD0FB6F894FA9AF99A0FBE2150D1
:101F000059F0F999FECF842F932F92BD81BDF89A95
:101F100080B5681739F7089582E00E94510F08953F
:101F2000A0E0B0E0E6E9FFE00C942821482E562E10
:101F3000EE24FF24C0E0D0E0CC24DD2488249924C2
:101F400004C055245394CC24DD24442051F46DEB7B
:101F5000E62E62E0F62EC0E0D0E05BE1852E912C0B
:101F600019C021E0421651F448EDE42E42E0F42E6F
:101F7000CDE1D0E039E2832E912C0CC032E0431643
:101F800049F42BE4E22E23E0F22EC8E4D0E090E204
:101F9000892E912C3E016C0C7D1C1092EE03109248
:101FA000ED03E3011BC0552059F4F999FECFD2BDD2
:101FB000C1BDF89A80B5F701E00FF11F808307C01B
:101FC000F701E00FF11FCE0160810E946E0F0E0D30
:101FD0001F1DF80180810E94C80021969E012619CC
:101FE000022F10E008151905F0F2CE015520D9F4A2
:101FF000F999FECFD2BDC1BDF89A20B5F999FECFAF
:102000002196D2BDC1BD2197F89A80B590E0B22E3D
:10201000AA248A299B292091ED033091EE032817E9
:10202000390759F48ECF21966091EE030E946E0F0E
:10203000CE016091ED030E946E0F80E091E0C80E2A
:10204000D91E91E0C91693E0D90608F47ECF852DFC
:10205000CDB7DEB7E0E10C94442182E060E00E945D
:10206000900F882331F48FEF9FEF90934C03809370
:102070004B03089582E061E00E94900F089597E07D
:102080009093BD0290E29093BE0291E29093BF02C2
:102090001092C00296E29093C1029093C20294E221
:1020A0009093C30295E29093C40292E09093CB0286
:1020B0009FEF9093CC022AE02093D5021092D60293
:1020C0001092D7021092CD021092CE021092CF023F
:1020D0001092D0029EE19093D1022093D20228EB7D
:1020E0003BE03093D4022093D302882361F080E058
:1020F00061E00E94900F8FEF9FEF90934C038093CD
:102100004B030E943A100895ADE5B0E0EAE8F0E133
:102110000C9426215B016C010E94741B1B012C0195
:1021200081E00E94160483E08093BC020E94390F74
:1021300084E894E06CE071E00E946A1E3E0108941D
:10214000611C711CE4C084E894E06AE171E00E94C3
:102150006A1E8FE70E94F1020E940503182F8983EF
:10216000823601F508ED12E00E940503F801819323
:102170008F01F3E001301F07B9F78091D802873350
:1021800009F0C0C084E894E063E271E00E946A1E36
:1021900082E48983CE01019661E00E94F7092C9ABE
:1021A00081E0CBC0803719F0893631F506C020E5D3
:1021B0002A83AA24BB24650105C081E00E943F1048
:1021C00089E48A838091EC03882321F08091CB02FB
:1021D000806803C08091CB028F778093CB02DE01B1
:1021E0001396EDEBF2E08BE101900D928150E1F757
:1021F000CE0102966CE184C08437E1F434E53E8F71
:1022000083E08F8F93E798A3E7E0E9A3FDE0FAA3CB
:10221000DE019396E6EDF1E08AE101900D928150A6
:10222000E1F7CE014E966FE10E94F709AA24BB2484
:10223000650168C0853791F40DEB12E00E9405033B
:10224000F80181938F01F2E0083D1F07B9F780E0A4
:1022500061E00E94900F25E5298350C0863631F554
:1022600080914B0390914C038F5F9F4FD1F086E498
:102270008DAF7BE4E72E73E0F72E8E01025C1F4FDB
:10228000F701819191917F010E947702F80190837B
:1022900081830E5F1F4FFBE6EF16F3E0FF0681F729
:1022A00001C01DAFCE01CD9661E22AC08736D9F4B8
:1022B0000BE413E00E940503982E88240E94050376
:1022C0009401280F311DC9010E944802F801819331
:1022D00091938F01F3E00B361F0761F727E4298301
:1022E0000E943A100BC0873469F48FEF9FEF9093F0
:1022F0004C0380934B030E943A101983C30161E0A1
:102300000E94F70993E09093BC020E94F504A11487
:10231000B104C104D10459F00E94741B62197309FD
:10232000840995096A157B058C059D0528F4809123
:10233000BC02843061F707CF80E0C35ADF4FE2E18F
:102340000C94422180E060E00E94900F882319F4F1
:1023500081E00E943F10089581E061E00E94900FAB
:10236000089581E060E00E94900F882311F490E0CE
:1023700006C090E08091D802873309F491E0892F5C
:102380000895EF92FF920F931F93CF93DF93EB018A
:102390009C01442737FD4095542F60E271EA87E0A5
:1023A00090E00E940B2189011216130614F001E03F
:1023B00010E0BE01882777FD8095982F20E231EA52
:1023C00047E050E00E94B6209801442737FD409531
:1023D000542F0E940B217901C0E0D0E009C0289A57
:1023E000C8010E94CC1B2898C8010E94CC1B2196D2
:1023F000CE15DF05A4F3CDB7DEB7E6E00C944E2191
:102400001F93182F2C9A83E00E94150380930103D9
:1024100084E00E9415038093020386E060E00E943E
:102420001B0387E061E00E941B0389E06FE70E94C5
:102430001B038AE065E00E941B038BE062E10E94BF
:102440001B038CE065E10E941B038DE06DEF0E9491
:102450001B038EE060E00E941B0380E76CE20E9499
:102460001B0380E360E00E941B0389E760E00E9499
:102470001B038AE765E00E941B0381E762E10E947B
:102480001B0382E762E00E941B0383E760E00E9477
:102490001B0384E760E00E941B036091CD027091F2
:1024A000CE028091CF029091D0020E94AC038DE6C3
:1024B00067E00E941B036AE070E080E090E00E9409
:1024C000A81B87E069E00E941B036AE070E080E0DF
:1024D00090E00E94A81B112369F010E007C088EB70
:1024E00091E061E070E00E94C111A8951F5F153175
:1024F000B1F74BC088E891E061E070E00E94C11143
:10250000A8958DE665E00E941B036AE070E080E01C
:1025100090E00E94A81B88EB91E061E070E00E94CF
:10252000C111A8958DE664E00E941B036AE070E08B
:1025300080E090E00E94A81B8DE591E061E070E0F2
:102540000E94C111A8958DE662E00E941B036AE01B
:1025500070E080E090E00E94A81B8FEA90E061E0CC
:1025600070E00E94C111A8958DE660E00E941B03F7
:102570006AE070E080E090E00E94A81B85E091E0B6
:1025800062E070E00E94C111A89587E061E00E94BE
:102590001B032C981F910895A6E1B0E0E2EDF2E153
:1025A0000C942821A8958CE00E941503882359F4E7
:1025B00084E894E06EE271E00E946A1E80E00E946E
:1025C00016040E94390F0E94F40D0E94821B0E9483
:1025D0001D0A90E0853009F491E08E010F5F1F4FD6
:1025E000BB24BA948091BC02843019F0992309F479
:1025F00088C10E94821B6B017C018091BC028430E7
:10260000F1F48FE70E94F10200E010E008C00E94A0
:102610000503F801E755FC4F80830F5F1F4F88EDDE
:1026200092E00E941E0190E00817190784F30E94AF
:10263000400390934303809342032C9A29C088ED72
:1026400092E00E941E01482F4F5F80E2B80121E016
:102650000E94E908882371F0B0926D030E94741BF8
:1026600060936E0370936F03809370039093710374
:1026700090E0B8CF88ED92E00E941E01482F29EA31
:1026800033E0FE013296C901BF0150E00E948C0088
:10269000C0922C03D0922D03E0922E03F0922F03D0
:1026A00010926C038091440390914503880F991F09
:1026B000816090934503809344032D9880E00E94AD
:1026C000830D8091A903282F30E0C9018E7390708B
:1026D000892B99F5F89480910003877062E672E087
:1026E0004AEA53E00E94AC010E949F0778948091CF
:1026F000A9039091730380FF1BC0992309F045C083
:10270000ABE4B3E020E030E0F901EE0FFF1FEE593B
:10271000FD4F808191818D939D932F5F3F4F20319D
:10272000310591F70E943A1081E0809373032DC028
:10273000992359F11092730328C0C90188739070CE
:10274000C89719F54091BE03842F822787FF1DC0CB
:1027500040584093BE038091C4028532B1F410E02A
:102760000AC01F5FE12FF0E0E755FC4F84E894E0DA
:1027700060810E942220212F30E08091A90390E007
:10278000877090708217930764F780916B0388239A
:1027900019F481E080936B0310924A03109248036E
:1027A0001092490380910003887109F4A1C04091FF
:1027B000BE038091A90390E0242F30E08227932765
:1027C00086FD60C0407C80E448274093BE03909122
:1027D000E7038091E803981701F1AFEBB3E030E035
:1027E0000FC03F5F892F90E0FC01E953FC4F20812F
:1027F0002D9301968F7190708093E703383031F0FC
:102800009091E7038091E803981759F7395C80911C
:10281000BE03382B3093BE0335C080913F038093B5
:10282000BF038091C102863251F482E10E94E01C14
:1028300095958795959587958093C00302C01092D2
:10284000C0038091C202863251F483E10E94E01CF1
:1028500095958795959587958093C10302C01092B1
:10286000C103809143038093C2038091420380930C
:10287000C30380914403909145039F770E949C027B
:102880008093C4038EEB93E069E00E94BB0902C011
:102890000E94F40D0E949E098823D1F30EEB12E0F2
:1028A00088E8E82E82E0F82EF8018081E82FF0E039
:1028B000CF01807F9070409791F4EF70F070EE0F31
:1028C000FF1FEE59FD4F8081918160E08F3F9105A0
:1028D00011F008F061E0F70180810E947D1C0F5F1C
:1028E0001F4F0894E11CF11CF2E0053C1F07E1F6C4
:1028F00083E08093BC020E94F50481E08093720320
:102900002C980E94821B5B016C010E94741B2B019E
:102910003C0180916C03823008F065C0E0902C038C
:10292000F0902D0300912E0310912F03809130031E
:1029300090913103A0913203B09133038E159F051E
:10294000A007B10709F44FC088ED92E00E9438015A
:10295000A60195012E193F09400B510B6C5D754086
:10296000804090406217730784079507E0F5E09276
:102970003003F092310300933203109333030E942B
:102980003C0380933F0320913D0330913E03280F89
:10299000311D30933E0320933D0360913C036F5FF4
:1029A00060933C036930F8F0C90170E00E94D520C3
:1029B000CB0170933E0360933D032091400343E0BD
:1029C000249F90011124820F931F969587959695C9
:1029D0008795809340030E949E0D10923E031092B3
:1029E0003D0310923C0380916B039090E903882390
:1029F00009F463C180906C03891408F0E1C188ED8B
:102A000092E00E94380120912C0330912D034091D7
:102A10002E0350912F03A21AB30AC40AD50A685193
:102A20007C4F8F4F9F4F6A157B058C059D0508F0E5
:102A300077C08091440390914503880F991F90932C
:102A400045038093440381E080937203882081F4DE
:102A500040923403509235036092360370923703EC
:102A6000109238031092390310923A0310923B03EC
:102A700080916C038F5F80936C0388ED92E00E94DD
:102A8000380120912C0330912D0340912E03509159
:102A90002F03260F371F481F591F20932C033093F5
:102AA0002D0340932E0350932F0381E080937203F4
:102AB0002D9A0E94830D0E949E0D32C088ED92E0F7
:102AC0000E9438019B01AC0180912C0390912D0351
:102AD000A0912E03B0912F0386017501E81AF90A1F
:102AE0000A0B1B0B682D70E080E090E00E94B6207E
:102AF0006E157F058007910798F410924503109298
:102B0000440381E080937203109240030E949E0D63
:102B1000A0922C03B0922D03C0922E03D0922F03CB
:102B200080916C03882309F4F2C09091D502992317
:102B300089F180914A03882369F5892F90E00E94EA
:102B4000E5002091340330913503409136035091D4
:102B5000370383017201E21AF30A040B150B6E1599
:102B60007F0580079107B0F481E080934A030E94BB
:102B7000DF078091D1020E941801640D751D861D2A
:102B8000971D6160609338037093390380933A0313
:102B900090933B039091D7029923F1F080914803E1
:102BA0008823D1F4892F90E00E94E500209134031E
:102BB0003091350340913603509137038301720100
:102BC000E21AF30A040B150B6E157F0580079107B7
:102BD00018F481E0809348039091D6029923F1F094
:102BE000809149038823D1F4892F90E00E94E50069
:102BF00020913403309135034091360350913703CF
:102C000083017201E21AF30A040B150B6E157F059E
:102C10008007910718F481E0809349038091CD02E9
:102C20009091CE02A091CF02B091D0020097A10561
:102C3000B10509F46CC08091380390913903A091DB
:102C40003A03B0913B030097A105B10509F45FC0B9
:102C500083017201E81AF90A0A0B1B0B17FD57C012
:102C60006091D20270E080E090E028EE33E040E036
:102C700050E00E94B6206E157F058007910708F08E
:102C800046C08091CB0290E0E4E096958795EA9566
:102C9000E1F781700E94001280E00E9416040E94F9
:102CA000F5040E94741B61606093380370933903CC
:102CB00080933A0390933B032AC088ED92E00E94F0
:102CC00038019B01AC0180912C0390912D03A091C0
:102CD0002E03B0912F0386017501E81AF90A0A0B39
:102CE0001B0B692D70E080E090E00E94B6206E150D
:102CF0007F058007910758F4A0922C03B0922D0312
:102D0000C0922E03D0922F0381E0809372038091B2
:102D100049038823B1F48091C402883219F40E94D7
:102D2000A90A0FC0893239F480914A0360916C037B
:102D30000E94860B06C08A3221F480914A030E94C9
:102D40001D0B809172038823B9F0E0912B03EF5F94
:102D5000E0932B03E83131F0F0E0E852FD4F878536
:102D6000882311F410922B0380912B030E942603D9
:102D70000E94450A1092720380916D038F3F21F5E6
:102D80000E94741B20916E0330916F034091700379
:102D900050917103621B730B840B950B695E73403A
:102DA0008040904088F00E94741B60936E03709383
:102DB0006F0380937003909371030E946E0A04C0A6
:102DC000891409F0ADCE7ACE6696E0E10C944421E8
:102DD000FF920F931F93082FF62E61E00E94111CA3
:102DE000802F61E00E947D1C8F2D61E00E947D1C80
:102DF0008AE090E00E94CC1B8F2D0E94B01C892B92
:102E000011F410E00FC0802F60E00E947D1C8AE06A
:102E100090E00E94CC1B8F2D0E94B01C10E0892BEB
:102E200009F411E0802F60E00E94111C802F60E007
:102E30000E947D1C8F2D60E00E947D1C812F1F91C0
:102E40000F91FF900895EF92FF920F931F937C01D3
:102E500004E814E0C8016F2D70E04AE050E00E94E1
:102E6000E71DC8016EE20E94261DB701E4E07695D9
:102E70006795EA95E1F76F707070C8014AE050E01D
:102E80000E94E71DC8016EE20E94261D8FE0E82225
:102E9000FF24C801B7014AE050E00E94E71D1F91DE
:102EA0000F91FF90EF900895A2E2B0E0EAE5F7E11C
:102EB0000C9426218E010F5F1F4F80E1D8011D92D7
:102EC0008A95E9F784E894E066E371E00E946A1E5F
:102ED0000E94390F20E431EE4DE958E12F8F38A3DD
:102EE00049A35AA380EC91EDA8E9BBE18B8F9C8F9D
:102EF000AD8FBE8F24EF31E040E050E02F8B388F54
:102F0000498F5A8F80E5C82E83ECD82EE12CF12C06
:102F1000B0E44B2EB1EE5B2EBDE96B2EB8E17B2EFB
:102F200088249924540133241E8A1D8A198A1A8AF6
:102F30001B8A1C8AFFC084E894E00E94E91F843445
:102F4000B9F0853430F48332B9F18C3209F0CCC059
:102F500044C0833509F0C8C02F8D38A149A15AA1BA
:102F6000C901DA012C013D01882499245401E2C0F1
:102F700084E894E064E40E94261D84E894E040E440
:102F800051EE6DE978E12AE030E00E940A1E84E803
:102F900094E06CE20E94261D84E894E040EC51ED40
:102FA00068E97BE12AE030E00E940A1E84E894E0B0
:102FB0006CE20E94441DBEC019821A821B821C82D0
:102FC0001D821E821F82188619861A861B861C8601
:102FD0001D861E861F86188A3AC0339434E0331645
:102FE00009F0A8C069817A818B819C8128EE33E049
:102FF00040E050E00E94B6206F8F78A389A39AA387
:103000006D817E818F8198850E94B6206B8F7C8F29
:103010008D8F9E8F89859A85AB85BC858F8B988F88
:10302000A98FBA8F6D857E858F8598890E94B6207D
:103030006B017C0190E2C9169EE4D90690E0E90696
:1030400090E0F90630F48CE162E30E941B03332424
:1030500071C0A0E3CA16A5E7DA06A0E0EA06A0E080
:10306000FA0618F48CE162E2F0CFB0E4CB16BCE9CA
:10307000DB06B0E0EB06B0E0FB0618F48CE166E29C
:10308000E4CFE0E5CE16E3ECDE06E0E0EE06E0E0BD
:10309000FE0618F48CE162E1D8CFF0E6CF16FAEE26
:1030A000DF06F0E0EF06F0E0FF0618F48CE165E1E2
:1030B000CCCF20E7C21621E1D20621E0E20620E0D3
:1030C000F20618F48CE161E0C0CF30EAC31636E8AE
:1030D000D30631E0E30630E0F30618F48CE163E058
:1030E000B4CF8CE165E0B1CFA0ED2A2E280E49E0E7
:1030F000421500F1032D10E0000F111F000F111FEA
:1031000081E090E08C0F9D1F080F191FD8016D9171
:103110007D918D919C912AE030E040E050E00E944A
:10312000B620620D711D811D911DF80160837183B0
:103130008283938384E894E00E94AF1F892B09F077
:10314000FACE81149104A104B10489F4C301B2013F
:103150000E94AC0361E070E080E090E00E94A81B58
:10316000FFEFFE8B1D8A198A1A8A1B8A1C8A2F89F7
:10317000388D498D5A8D82169306A406B506E0F463
:103180000E943C0329893A894B895C89280F311DAB
:10319000411D511D298B3A8B4B8B5C8B3D89381718
:1031A00008F48D8B4E89841708F48E8B0894811C4B
:1031B000911CA11CB11C56C0C301B20128EE33E022
:1031C00040E050E00E94E92084E894E0BA01A901BF
:1031D0002AE030E00E94D81D84E894E06CE20E946E
:1031E000261D84E894E06D894AE050E00E94F81DB5
:1031F00084E894E06CE20E94261D69897A898B89B3
:103200009C89A50194010E94E92084E894E0BA0118
:10321000A9012AE030E00E94D81D84E894E06CE225
:103220000E94261D84E894E06E894AE050E00E94E6
:10323000F81D84E894E06CE20E94441D4C0C5D1C77
:103240006E1C7F1C8B8D9C8DAD8DBE8D8415950560
:10325000A605B70520F44F8C58A069A07AA0882451
:10326000992454012F8D38A149A15AA1285E3340D9
:103270004040504009F05ECFA296E2E10C9442211A
:1032800080E065E970E042E050E00E94AF1A0895E6
:10329000A1E0B0E0EEE4F9E10C94362180E00E9478
:1032A000B1008CE061E00E94111C8DE061E00E94A1
:1032B000111C0E94240F80E060E00E94111C81E03C
:1032C00061E00E94111C84E894E040E052EC61E06F
:1032D00070E00E94281F0E94A2110E942D1084E815
:1032E00094E063E471E00E94671E83E793E00E942C
:1032F000231784E894E06AE571E00E94671E84E881
:1033000094E062E070E04AE050E00E94531E0E94A8
:10331000401978942D9A8EE062E10E94E816882385
:1033200029F02D982C980E945417FBCF8AE063E077
:103330000E94E816882329F40E94B111882309F01D
:1033400006C184E894E062E671E00E94671E60E0D6
:1033500070E080E090E00E948410882349F00E9491
:10336000AC1184E894E06BE971E00E946A1E2C9A2B
:103370000E941E0E22C08091C202833229F08091E9
:10338000CB028B7F8093CB028091CB0281FF15C053
:1033900082FD13C064EF71E080E090E00E94841031
:1033A000882359F00E94AC1184E894E06BE971E045
:1033B0000E946A1E0E941E0E2C9A8091C1028232C7
:1033C00039F58091C202833219F581E00E94D70D50
:1033D0008091CB0282FF09C084E894E066EB71E043
:1033E0000E946A1E0E946C0813C064E170E080E0D5
:1033F00090E00E94A81B80E2BE016F5F7F4F41E01A
:1034000021E00E94E908882319F481E080936D038C
:1034100084E894E061EC71E00E94671E8FE00E94F6
:10342000B10080E00E94160410922B0380E00E94FD
:1034300026031092E90390E0983158F4292F2F5F6A
:10344000E92FF0E0E852FD4F8785882311F0922F95
:10345000F3CF9093E90383E08093BC020E94390F7D
:1034600080916D03882311F00E946E0A8091C4023E
:10347000883211F08A3239F484E894E040E052EC6A
:1034800061E070E02BC0893271F484E894E040EA96
:1034900056E861E070E00E94281F8091C2008062BF
:1034A0008093C20022C0809100038871803169F04E
:1034B0004091D9025091DA026091DB027091DC02F6
:1034C0004A3051056105710538F484E894E040E81C
:1034D00055E260E070E002C084E894E00E94281F9A
:1034E00004C084E894E00E94E91F84E894E00E940C
:1034F000AF1F892BB1F78091C302843229F08091EC
:10350000C1008F7E8093C1008091C402853259F042
:103510008A3249F0893239F0883229F08091C1002D
:10352000877F8093C1001092E7031092E803109206
:103530006B030E94821B60932C0370932D03809376
:103540002E0390932F032196E2E00C9452210E94C7
:103550001E0E8091C102823209F011CF0CCF823051
:1035600000F5E82FF0E0EE0FFF1FE151FC4F7183F3
:103570006083882319F08130A1F408C0809169002C
:103580008C7F842B80936900E89A0895809169006C
:10359000440F551F440F551F837F842B8093690070
:1035A000E99A08951F920F920FB60F9211242F934C
:1035B0003F934F935F936F937F938F939F93AF93BB
:1035C000BF93EF93FF938091EF039091F003892BCA
:1035D00029F0E091EF03F091F0030995FF91EF914D
:1035E000BF91AF919F918F917F916F915F914F911B
:1035F0003F912F910F900FBE0F901F9018951F9223
:103600000F920FB60F9211242F933F934F935F9316
:103610006F937F938F939F93AF93BF93EF93FF939A
:103620008091F1039091F203892B29F0E091F1034D
:10363000F091F2030995FF91EF91BF91AF919F91A6
:103640008F917F916F915F914F913F912F910F904B
:103650000FBE0F901F9018951F920F920FB60F92EA
:1036600011242F933F938F939F93AF93BF93809198
:10367000F7039091F803A091F903B091FA03309108
:10368000FB030196A11DB11D232F2D5F2D3720F0C7
:103690002D570196A11DB11D2093FB038093F703C5
:1036A0009093F803A093F903B093FA038091F30386
:1036B0009091F403A091F503B091F6030196A11D3A
:1036C000B11D8093F3039093F403A093F503B0939B
:1036D000F603BF91AF919F918F913F912F910F90E2
:1036E0000FBE0F901F9018958FB7F8942091F70395
:1036F0003091F8034091F9035091FA038FBFB9015B
:10370000CA0108959FB7F8942091F3033091F40310
:103710004091F5035091F60386B5A89B06C08F3FF4
:1037200021F02F5F3F4F4F4F5F4F9FBF542F432FCD
:10373000322F2227280F311D411D511D82E0220FFB
:10374000331F441F551F8A95D1F7B901CA01089547
:10375000EF92FF920F931F93CF93DF937B018C0126
:103760000E94821BEB010EC00E94821B6C1B7D0B12
:10377000685E7340C8F30894E108F1080109110973
:10378000C851DC4FE114F1040105110569F7CDB70B
:10379000DEB7E6E00C944E21019739F0880F991FAF
:1037A000880F991F02970197F1F70895789484B5CF
:1037B000826084BD84B5816084BD85B5826085BD2D
:1037C00085B5816085BDEEE6F0E080818160808313
:1037D000E1E8F0E0108280818260808380818160F6
:1037E0008083E0E8F0E0808181608083E1EBF0E0BD
:1037F000808184608083E0EBF0E080818160808361
:10380000EAE7F0E080818460808380818260808349
:103810008081816080838081806880831092C10074
:103820000895CF93DF93482F50E0CA0186569F4FEB
:10383000FC0134914A575F4FFA018491882369F162
:1038400090E0880F991FFC01E859FF4FA591B491B2
:10385000FC01EE58FF4FC591D491662351F42FB768
:10386000F8948C91932F909589238C938881892348
:103870000BC0623061F42FB7F8948C91932F909520
:1038800089238C938881832B88832FBF06C09FB7A1
:10389000F8948C91832B8C939FBFDF91CF910895E7
:1038A000833071F0843028F48130A1F0823021F52A
:1038B00014C08630B1F08730D1F08430E9F404C010
:1038C000809180008F7703C0809180008F7D8093EE
:1038D0008000089584B58F7702C084B58F7D84BD44
:1038E00008958091B0008F778093B0000895809103
:1038F000B0008F7D8093B0000895FF920F931F93C7
:10390000F62E482F50E0CA0182559F4FFC012491AA
:10391000CA0186569F4FFC0114914A575F4FFA0126
:1039200004910023C9F0222319F0822F0E94501C19
:10393000E02FF0E0EE0FFF1FEE58FF4FA591B4917E
:103940009FB7F894FF2021F48C911095812302C039
:103950008C91812B8C939FBF1F910F91FF900895A5
:103960000F931F93482F50E0CA0182559F4FFC01CF
:103970002491CA0186569F4FFC0104914A575F4F1C
:10398000FA011491112319F420E030E015C022232C
:1039900019F0822F0E94501C812F90E0880F991FF0
:1039A00084589F4FFC01A591B4918C9120E030E0A8
:1039B000802311F021E030E0C9011F910F9108959B
:1039C000982F8E3008F09E509770809187028295D4
:1039D000880F880F807C892B80937C0080917A00EF
:1039E000806480937A0080917A0086FDFCCF2091DC
:1039F000780040917900942F80E030E0282B392B1B
:103A0000C9010895A0E0B0E0E8E0FDE10C943021A8
:103A10007C016B018A01C0E0D0E00FC0D6016D913E
:103A20006D01D701ED91FC910190F081E02DC7016E
:103A30000995C80FD91F015010400115110571F7E4
:103A4000CE01CDB7DEB7E8E00C944C21DC01ED915E
:103A5000FC910190F081E02D09950895EF92FF927D
:103A60000F931F938C016DE00E94261D7C01C801FD
:103A70006AE00E94261D9C012E0D3F1DC9011F9169
:103A80000F91FF90EF900895EF92FF920F931F9385
:103A90007C010E94261D8C01C7010E942E1D9C01E5
:103AA000200F311FC9011F910F91FF90EF900895D2
:103AB000CF93DF93EC016115710519F420E030E03C
:103AC0000FC0DB010D900020E9F71197A61BB70B83
:103AD000E881F9810280F381E02DAD0109959C0117
:103AE000C901DF91CF9108954F925F927F928F929B
:103AF0009F92AF92BF92CF92DF92EF92FF920F937D
:103B00001F93DF93CF93CDB7DEB7A1970FB6F8948D
:103B1000DEBF0FBECDBF2C01742ECB01223008F4C6
:103B20002AE019A231E2C32ED12CCC0EDD1E822E4A
:103B30009924AA24BB24672D752FA50194010E9406
:103B4000E92079018A01C801B701A50194010E9409
:103B5000B620472D461B0894C108D1084A3010F4FE
:103B6000405D01C0495CF6014083E114F1040105A8
:103B7000110521F07E2C5F2DC801DDCFC201B601F9
:103B80000E94581DA1960FB6F894DEBF0FBECDBFA0
:103B9000CF91DF911F910F91FF90EF90DF90CF9029
:103BA000BF90AF909F908F907F905F904F900895BF
:103BB000DC012115310541F4ED91FC910190F0817A
:103BC000E02D642F099508950E94741D0895EF92C9
:103BD000FF920F931F939A017B0100E010E0B80160
:103BE000A7010E94D81D1F910F91FF90EF9008959B
:103BF000EF92FF920F931F939A01E62EFF2400E0AD
:103C000010E0B801A7010E94D81D1F910F91FF90ED
:103C1000EF900895A0E0B0E0E0E1FEE10C943021E7
:103C2000EC016A017B012115310541F4E881F9813C
:103C30000190F081E02D642F09951BC02A303105D9
:103C4000B1F477FF13C06DE20E94261D8C0144275A
:103C50005527BA014C195D096E097F09CE012AE08A
:103C60000E94741D9C01200F311F04C02AE00E9495
:103C7000741D9C01C901CDB7DEB7E8E00C944C215E
:103C8000EF92FF920F931F937B019A010027F7FC9D
:103C90000095102FB801A7010E940A1E1F910F91D5
:103CA000FF90EF900895EF92FF920F931F937C0186
:103CB0000E94401E8C01C7010E942E1D9C01200FF6
:103CC000311FC9011F910F91FF90EF9008950E943D
:103CD000581D0895EF92FF920F931F937C010E944D
:103CE000671E8C01C7010E942E1D9C01200F311FF1
:103CF000C9011F910F91FF90EF90089508951F92B1
:103D00000F920FB60F9211242F933F934F938F93DF
:103D10009F93EF93FF938091C00082FD1DC040915F
:103D2000C60020913C0430913D042F5F3F4F2F731C
:103D3000307080913E0490913F042817390771F04C
:103D4000E0913C04F0913D04E450FC4F40833093FB
:103D50003D0420933C0402C08091C600FF91EF9186
:103D60009F918F914F913F912F910F900FBE0F9088
:103D70001F9018951F920F920FB60F9211242F9338
:103D80003F938F939F93EF93FF9320918004309103
:103D9000810480918204909183042817390731F4BB
:103DA0008091C1008F7D8093C10014C0E091820496
:103DB000F0918304E05CFB4F20818091820490911C
:103DC000830401968F739070909383048093820490
:103DD0002093C600FF91EF919F918F913F912F917A
:103DE0000F900FBE0F901F901895A0E0B0E0EBEF82
:103DF000FEE10C942C21FC011382128288EE93E0E8
:103E0000A0E0B0E084839583A683B78380EB92E043
:103E1000918380837587648757874687318B208B92
:103E2000138B028BF58AE48AD78AC68AB18EA08E5C
:103E3000938E828E8F85848F8889858F8989868FDE
:103E40008A89878F8B8980A32096ECE00C94482187
:103E5000AF92BF92DF92EF92FF920F931F93CF9397
:103E6000DF93EC017A018B01DD24403081EE5807AD
:103E700080E0680780E0780711F0DD24D39491E0BA
:103E8000A92EB12CEC89FD89DD2069F0C50108A0BF
:103E900002C0880F991F0A94E2F7808360E079E0FE
:103EA0008DE390E005C0108260E874E88EE190E058
:103EB000A80197010E94E920215030404040504025
:103EC000569547953795279580E12030380720F0A3
:103ED000DD2011F0DD24D6CFE889F9893083EA8925
:103EE000FB89208319A2EE89FF89408121E030E01F
:103EF000C9010C8C02C0880F991F0A94E2F7482B65
:103F00004083EE89FF894081C9010D8C02C0880F72
:103F1000991F0A94E2F7482B4083EE89FF8940817C
:103F2000C9010E8C02C0880F991F0A94E2F7482B32
:103F30004083EE89FF8980810F8C02C0220F331FDE
:103F40000A94E2F7209528232083DF91CF911F91D7
:103F50000F91FF90EF90DF90BF90AF900895DC013C
:103F60001C96ED91FC911D97E05CFF4F21913191E2
:103F700080819181281B390B2F733070C9010895FE
:103F800084E894E00E94AF1F892B11F00E947E1EEE
:103F90000895DC011C96ED91FC911D97E05CFF4FAC
:103FA00020813181E054F040DF01AE5BBF4F8D9145
:103FB0009C9111972817390719F42FEF3FEF07C08D
:103FC0008D919C91E80FF91F8081282F30E0C90165
:103FD0000895DC011C96ED91FC911D97E05CFF4F6C
:103FE00020813181E054F040DF01AE5BBF4F8D9105
:103FF0009C9111972817390719F42FEF3FEF10C044
:104000008D919C911197E80FF91F20818D919C91C2
:10401000119701968F73907011969C938E9330E058
:10402000C9010895DC0191968C919197882339F00C
:104030005496ED91FC915597808186FFF9CF91962A
:104040001C920895CF93DF93EC01EE85FF85E05C31
:10405000FF4F20813181E054F0402F5F3F4F2F739D
:104060003070DF01AE5BBF4F8D919C911197281787
:104070003907D1F3E05CFF4F80819181E054F0403B
:10408000E80FF91F6083EE85FF85E05CFF4F318309
:104090002083EE89FF89208181E090E00F8C02C0AF
:1040A000880F991F0A94E2F7282B208381E089A3C7
:1040B000EC89FD8980818064808381E090E0DF91DC
:1040C000CF9108958F929F92AF92BF92CF92DF923D
:1040D000EF92FF920F931F9300D000D00F92EDB795
:1040E000FEB7319684E0ADB7BEB711968C9383E0EE
:1040F000818387E0828385E0838381E0848384E811
:1041000094E06CEF73E040E454E025EC30E004EC24
:1041100010E0B0ECEB2EF12CA1ECCA2ED12CF2EC7D
:10412000AF2EB12CE6EC8E2E912C0E94F51E0F9036
:104130000F900F900F900F901F910F91FF90EF90A5
:10414000DF90CF90BF90AF909F908F900895CF93C6
:10415000DF930E94D61B0E944819C0ECDFE10E9449
:10416000CC122097E1F30E94C01FF9CF629FD001CB
:10417000739FF001829FE00DF11D649FE00DF11D22
:10418000929FF00D839FF00D749FF00D659FF00DD1
:104190009927729FB00DE11DF91F639FB00DE11DBE
:1041A000F91FBD01CF0111240895AA1BBB1B51E1CA
:1041B00007C0AA1FBB1FA617B70710F0A61BB70B97
:1041C000881F991F5A95A9F780959095BC01CD013C
:1041D0000895A1E21A2EAA1BBB1BFD010DC0AA1F48
:1041E000BB1FEE1FFF1FA217B307E407F50720F060
:1041F000A21BB30BE40BF50B661F771F881F991FDB
:104200001A9469F760957095809590959B01AC0123
:10421000BD01CF01089597FB092E05260ED057FD4D
:1042200004D0D7DF0AD0001C38F450954095309563
:1042300021953F4F4F4F5F4F0895F6F7909580952A
:10424000709561957F4F8F4F9F4F08952F923F92AA
:104250004F925F926F927F928F929F92AF92BF9296
:10426000CF92DF92EF92FF920F931F93CF93DF9342
:10427000CDB7DEB7CA1BDB0B0FB6F894DEBF0FBE9F
:10428000CDBF09942A88398848885F846E847D84EC
:104290008C849B84AA84B984C884DF80EE80FD80EE
:1042A0000C811B81AA81B981CE0FD11D0FB6F89464
:1042B000DEBF0FBECDBFED010895EE0FFF1F0590CD
:0A42C000F491E02D0994F894FFCF6B
:1042CA0054582074696D656F75742100576169745B
:1042DA00696E672062696E640A00476F7420706BAA
:1042EA00740A006461746120676F6F640A0052582F
:1042FA002068616E67007363616E6E6572206D6F10
:10430A006465004F70656E4C52536E672052582098
:10431A007374617274696E672000206F6E2048574B
:10432A002000454550524F4D2064617461206E6FE4
:10433A00742076616C6964206F722062696E6420F1
:10434A006A756D70706572207365742C20666F7261
:10435A0063696E672062696E640A005361766564F8
:10436A002062696E64206461746120746F2045451F
:10437A0050524F4D0A004920616D20736C61766579
:10438A0000456E746572696E67206E6F726D616C3E
:10439A00206D6F646500002001270121022B032292
:1043AA000326042304260524062506280629062AA8
:1043BA00C01200001A400AA1204EA5001B1E275257
:1043CA002C23308025000005400AA1204EA500209C
:1043DA00244EA52C2330004B000006400AD0009D35
:1043EA0049007B289D492C233000E1000005400A42
:1043FA004501D7DC03B81E0EBF00232E48E8010092
:10440A008A400A6001555502AD1E20000023C8806B
:10441A0025000005400AA1204EA50020244EA52C07
:10442A002330000200020002000200020002000221
:10443A000002000200020002000200020002000262
:10444A0000028813409C08010A030E12130001049B
:10445A000000000008000100001000002000000019
:10446A000100000200070B0C1011150000000000EB
:0C447A002220021DAF1FE91FC91F1220E5
:107E00000F92CDB7DEB7112484B714BE81FFF1D035
:107E100082E08093C00088E18093C10086E0809377
:107E2000C20080E18093C4008EE0CDD088249924E4
:107E3000CC24C394F5E0DF2EE1E1EE2E73E0F72EC3
:107E4000B6D0082F813479F4B2D08983C2D0898129
:107E5000823811F481E005C0813811F485E001C059
:107E600083E09ED09AC0823411F484E103C085344B
:107E700019F485E0B6D091C0853561F498D0082F0B
:107E800010E095D090E0982E8824802A912A880CC2
:107E9000991C82C0863521F484E0A3D080E0E1CF34
:107EA000843609F04CC083D082D0A82E80D0B82E62
:107EB00000E011E07CD0F80181938F01AE16D1F77C
:107EC00088D0FB2DF53489F4E0E0F1E00BC0F9999E
:107ED000FECF92BC81BC0894811C911C819180BD15
:107EE000FA9AF99AEA1598F358C08B2D863409F05E
:107EF00054C0F401F7BEE89507B600FCFDCFF401CD
:107F0000A0E0B1E02C9130E011968C91119790E0B7
:107F1000982F8827822B932B12960C01C7BEE895C9
:107F20001124329681E0A038B80761F7F401D7BE7A
:107F3000E89507B600FCFDCFE7BEE8952EC0843774
:107F4000F1F435D034D0182F32D0B82E42D0FB2DDA
:107F5000F63421F4F40105914F010CC0FB2DF534EA
:107F600049F4F999FECF92BC81BC0894811C911C04
:107F7000F89A00B5802F14D0115049F70EC08537FC
:107F800039F427D08EE10CD085E90AD08FE069CF93
:107F9000813511F488E017D01CD080E101D050CF9A
:107FA0009091C00095FFFCCF8093C600089580910A
:107FB000C00087FFFCCF8091C00084FD01C0A89560
:107FC0008091C6000895E0E6F0E098E19083808318
:107FD0000895EDDF803219F088E0F5DFFFCF84E10E
:107FE000DFCF1F93182FE3DF1150E9F7F2DF1F9166
:0E7FF0000895282E80E0E7DFEE27FF27099492
:027FFE0001057B
:0400000300007E007B
:00000001FF
